:10000000000018308A00722EFF00030E8301A10049
:100010000A08A0008A010408A2007708A300780853
:10002000A4007908A5007A08A6007B08A70083131E
:1000300083128C308400801E1F288C1A38288C3044
:100040008400001C25280C183B2822088400230863
:10005000F7002408F8002508F9002608FA00270808
:10006000FB0020088A00210E8300FF0E7F0E09008E
:100070008A110A127D288A110A12FC280A108A1095
:100080000A11820731342E343034003464008C1E5F
:1000900046281808E8001A08F800E81C5128181229
:1000A00018160034F701F8018316031758080310D7
:1000B0005918F707F70CF80CD918F707F70CF80CD4
:1000C0005919F707F70CF80CD919F707F70CF80CC2
:1000D000591AF707F70CF80CD91AF707F70CF80CB0
:1000E000591BF707F70CF80CD91BF707F70CF80C9E
:1000F000031383128A110A12E028A0306A078400D1
:10010000831383160317D9010408D8005910831BE1
:1001100059148312031346208316031758088400CA
:1001200083135918831778088000A03083120313B3
:100130006A078400831300082F3C031DB32866154B
:10014000EA0183160317D50155080B3C031CAF28A1
:10015000A0305507840083138001D50AA4282F30CE
:100160000313A0008312661DF828A0306A078400DC
:10017000831300080D3C031DF0286A08043C031893
:10018000F0286611EA010130E900831621082F3CAE
:100190000318EE282108393C031CEE2822082F3CC6
:1001A0000318EE282208393C031CEE2830302102C7
:1001B0000317D700D8000A30D9008312031352283E
:1001C000780883160317D800303003132202031770
:1001D000580783120313EC00F02883168312E901F9
:1001E0000130EA076A080C3C0318F8286611EA0196
:1001F0008C128A110A1225282030F8001F08C739EE
:1002000078049F001F15F6308F0041308E00670B79
:100210000B29E7010D290130E700E708031D12292A
:10022000871013298714EF106F0883168700831235
:100230001F1918291E08FA0083161E080317D50077
:100240007A08D60083120313430883160317560255
:10025000031C4129031D3729550883120313420249
:10026000031C3529831603174129831603178312AC
:1002700003133C1607156F116F0883168700482972
:1002800003178312031307116F116F08831687007A
:1002900083120C108A110A1225280C30F70007303F
:1002A00081018130840083130008F0390738800011
:1002B00064000008F739F719F03977048000B53089
:1002C00090008A150A16DB2E031738088D00831656
:1002D0008C130C1483120C08F8000313003403175A
:1002E0003408B40AB700B800031364217808031770
:1002F000B5003408B8000313642178080317B6006A
:100300003508F8003608F9000313003403173908DC
:100310008D003A088C0083168C130C15831203137E
:100320000B08F7008B138316031755308D00AA3086
:100330008D008C148C189A290C11770883120313E2
:100340008B04003403173408B40AB7003508B8002A
:100350003708B9003508BA00031386210317360899
:10036000B7003408B9003608BA00031386210034F8
:1003700020300317CB00C701C801C901CA014208D8
:10038000FA004108F9004008F8003F08F7000310A0
:10039000771CD8294308C70744080318440FC80727
:1003A00045080318450FC90746080318460FCA0732
:1003B000CA0CC90CC80CC70CFA0CF90CF80CF70CD9
:1003C000CB0BC72903130034F701F801F901FA0137
:1003D0000317C901CA01CB01CC01480847044604F0
:1003E00045040319232A2030CD000310C10DC20D8E
:1003F000C30DC40DC90DCA0DCB0DCC0D48084C0260
:10040000031D0C2A47084B02031D0C2A46084A020A
:10041000031D0C2A45084902031C1D2A4508C90270
:100420004608031C460FCA024708031C470FCB02AD
:100430004808031C480FCC020314F70DF80DF90D02
:10044000FA0DCD0BF52949308400831703130034CE
:10045000031793019201031332080317910003134A
:100460003108031790001308C2001208C1001108D8
:10047000C0001008BF00C601C501C401C830C300D8
:100480000313B8217A0803179400790893007808B9
:100490009200770891001408C2001308C1001208E6
:1004A000C0001108BF00C601C501C4010530C3006A
:1004B0000313B8217A080317950079089400780887
:1004C00093007708920096004030130797001408B5
:1004D00098001F3003182030980715089900003045
:1004E0000318013099079D01190C9C00180C9B0002
:1004F000170C9A009C0C9B0C9A0C9C0C9B0C9A0C55
:100500009C0C9B0C9A0C0F309C051D08C2001C080B
:10051000C1001B08C0001A08BF00C601C501033096
:10052000C400FF30C3000313B8217A0803179E00EC
:1005300079089D0078089C0077089B001E08C4007D
:100540001D08C3001C08C2001B08C100C801C70168
:100550000330C600E830C5000313E4217808C30067
:100560007708C20000340317930192010313300887
:100570000317910003132F08031790001308C200FC
:100580001208C1001108C0001008BF00C601C50153
:10059000C401C830C3000313B8217A0803179400BC
:1005A0007908930078089200770891001408C20037
:1005B0001308C1001208C0001108BF00C601C50120
:1005C000C4010530C3000313B8217A08031795004E
:1005D00079089400780893007708920096004030DC
:1005E00013079700140898001F300318203098074D
:1005F0001508990000300318013099079D01190C66
:100600009C00180C9B00170C9A009C0C9B0C9A0CDD
:100610009C0C9B0C9A0C9C0C9B0C9A0C0F309C0510
:100620001D08C2001C08C1001B08C0001A08BF003A
:10063000C601C5010330C400FF30C3000313B82155
:100640007A0803179E0079089D0078089C007708B7
:100650009B001E08C4001D08C3001C08C2001B0824
:10066000C100C801C7010330C600E830C50003134C
:10067000E4217808C5007708C40000349412EF1212
:100680006F088316870083126F166F088316870022
:100690008312EF156F0883168700253083129400AC
:1006A0000030831694002F308500C030860019304A
:1006B00087008312EF00051283160512831286123B
:1006C000831686128312061283160612831286116F
:1006D0008316861183120611831606118312861063
:1006E0008316861083120610831606108312871055
:1006F000EF106F0883168700831207116F116F08C0
:100700008316870083128712EF126F088316870003
:10071000831207136F136F088316870083128713E2
:10072000EF136F08831687001F1383121F179F177D
:1007300083169F1783121F1483161F109F101F11FB
:100740009F150730831203178D0083168C130C142A
:1007500083120C08993C031DC82BB40103136F21AD
:100760007908B0007808AF0002300317B400031313
:100770006F217908B2007808B10004300317B40083
:1007800003136F217908B4007808B300262C0317EF
:10079000B401031330080317B60003132F0803171F
:1007A000B5000313A22102300317B400031332086B
:1007B0000317B600031331080317B5000313A22172
:1007C00004300317B400031334080317B6000313EF
:1007D00033080317B5000313A2210317B401031351
:1007E0006F217908FA0078082F02031D192C7A0866
:1007F0003002031D192C02300317B40003136F21BC
:100800007908FA0078083102031D192C7A0832029F
:10081000031D192C04300317B40003136F2179084A
:10082000FA0078083302031D192C7A0834020319E0
:100830001B2C3C14262C9930B60007300317B90046
:10084000031336080317BA0003138621BD1E292C93
:10085000BD142822B322C0308B0483160C130C1451
:1008600083128A150A12F428903084008317000836
:1008700003194B2C0130F800BF30F7006400F70B70
:100880003E2CF80B3C2C4A30F700F70B452C0000AF
:100890006400800B3A2C00341F151F194D2C831651
:1008A0001E088312BE001E08BF00C001C10141081E
:1008B0000317C200031340080317C10003133F08C6
:1008C0000317C00003133E080317BF00C601C5018C
:1008D0000330C400E830C3000313B8217A080317BB
:1008E000B9007908B8007808B7007708B600390869
:1008F000C4003808C3003708C2003608C100C80168
:10090000C7010330C600FF30C5000313E4217A0895
:100910000317BA007908B9007808B8007708B7005B
:100920003408F7003508F800F901FA017A08BE002A
:100930007908BD003508BC003408BB003A08C20085
:100940003908C1003808C0003708BF003E08C6009B
:100950003D08C5003508C4003408C3000313B8219E
:100960007A08C1007908C0007808BF007708BE0087
:1009700000346D08840083136E188317031763080F
:100980008000840A80010313ED0A0319EE0A003483
:1009900004080317B9003B30C0009A30BF00CA30CA
:1009A000BE00BD010A30BB003808031DB90337087B
:1009B000C4003608C3003508C2003408C10040082E
:1009C000C8003F08C7003E08C6003D08C500031325
:1009D000E42100080317B400840A0008B500840A63
:1009E0000008B600840A0008B700FD308407F70845
:1009F000031D0D2D380A3B0203190D2D390803196B
:100A00000E2D0F393B020319072D0318252DB91B95
:100A1000252D391B0E2D20301F2DB90138083B0222
:100A2000031D1E2D7708B9002E30E3000313B924EF
:100A300003173908F7002030B90500303030F707C8
:100A40007708E3000313B92403174008C4003F08E4
:100A5000C3003E08C2003D08C100C801C701C6016D
:100A60000A30C5000313E4217A080317C00079088F
:100A7000BF007808BE007708BD00BB0BD72C03135E
:100A800000340317B6013508FA00340884008313D4
:100A90007A188317800803196A2D36080A3C031C4C
:100AA0006A2D3508FA003408B40A0319B50A84001F
:100AB00083137A1883170008B7000313130803176A
:100AC0003708031393008316141C642D8312031735
:100AD000B60A432D031300341F151F196D2D8316FD
:100AE0001E088312BE001E08BF00C001C1014108DC
:100AF0000317C200031340080317C10003133F0884
:100B00000317C00003133E080317BF00C601C50149
:100B10000330C400E830C3000313B8217A08031778
:100B2000BD007908BC007808BB007708BA003D0812
:100B3000C4003C08C3003B08C2003A08C100C80119
:100B4000C7010330C600FF30C5000313E4217A0853
:100B50000317BE007908BD007808BC007708BB0009
:100B60003E08C2003D08C1003C08C0003B08BF0071
:100B7000C601C5013708C4003608C3000313B821F5
:100B80007A08C1007908C0007808BF007708BE0065
:100B9000BE08031DD52DBF08031DD52DC008031D9C
:100BA000D52DC108031DD52D482E0317BD01BC014D
:100BB0003508BB003408BA003D08C2003C08C1003B
:100BC0003508C0003408BF00C601C5010330C400A9
:100BD000E830C3000313B8217A080317BE00790870
:100BE000BD007808BC007708BB0003103E0CFA007B
:100BF0003D0CF9003C0CF8003B0CF7000313BE025F
:100C00007808031C780FBF027908031C790FC00213
:100C10007A08031C7A0FC10241080317C4000313AA
:100C200040080317C30003133F080317C200031350
:100C30003E080317C100C801C701C6013908C50035
:100C40000313E4217A08C1007908C0007808BF00C6
:100C50007708BE0041080317C400031340080317B8
:100C6000C30003133F080317C20003133E08031712
:100C7000C100C801C701C6013808C5000313E4213B
:100C80007A08C1007908C0007808BF007708BE0064
:100C900000340317920183160313141C4D2E831284
:100CA0000317120810078400831311188317031306
:100CB00013088000003A03196C2E031712080A3C2F
:100CC0000318642E03136C2E920A64001030F70090
:100CD000F70B682E512E031300340317BD01BB011F
:100CE0000A30BC00BA01B901B801B70135083604B1
:100CF000031D7F2EF701F801F901FA01D92F3D08F4
:100D0000BD0A350784008313361883170008BE0018
:100D10003E082D3C031D982E0130BB003D08BD0A46
:100D2000350784008313361883170008BE00A52EEC
:100D30003E082B3C031DA52E3D08BD0A3507840047
:100D40008313361883170008BE003E082F3C031893
:100D5000C02F3E08393C031CC02F3E08303C031D09
:100D6000D12E3D08350784008313361883170008F9
:100D7000783C0319C52E3D083507840083133618C7
:100D800083170008583C031DD12E1030BC00BD0A4B
:100D90003D08BD0A35078400831336188317000801
:100DA000BE003C080A3C031D272F3E082F3C0318B9
:100DB000262F3E08393C031C262F0310370DC00098
:100DC000380DC100390DC2003A0DC300370DF700D0
:100DD000380DF800390DF9003A0DFA00F70DF80D4D
:100DE000F90DFA0DF70DF80DF90DFA0DF830F705BC
:100DF00077084007B7004108B80078080318780F53
:100E0000B8074208B90079080318790FB9074308F1
:100E1000BA007A0803187A0FBA0730303E02B707D3
:100E2000003003180130B807003003180130B9074B
:100E3000003003180130BA073D08BD0A35078400A9
:100E40008313361883170008BE00D52EC02F3C0828
:100E5000103C031DC02F3E08603C0318362F3E088F
:100E60007A3C031C362F3E08DF39372F3E08BE0080
:100E70003E082F3C0318402F3E08393C0318482FEA
:100E80003E08403C0318C02F3E08463C031CC02FC0
:100E90003E082F3C03187D2F3E08393C031C7D2F54
:100EA000370DC000380DC100390DC2003A0DC30026
:100EB000C00DC10DC20DC30DC00DC10DC20DC30DBE
:100EC000C00DC10DC20DC30DF030C00530303E0263
:100ED0004007B7004108B800003003180130B807D8
:100EE0004208B900003003180130B9074308BA00BE
:100EF000003003180130BA07AA2F370DC000380D93
:100F0000C100390DC2003A0DC300C00DC10DC20DA4
:100F1000C30DC00DC10DC20DC30DC00DC10DC20D5D
:100F2000C30DF030C00541303E020A3E4007B70015
:100F30004108B800003003180130B8074208B90072
:100F4000003003180130B9074308BA000030031815
:100F50000130BA073D08BD0A3507840083133618EF
:100F600083170008BE00603C0318BD2F3E087A3C82
:100F7000031CBD2F3E08DF39BE2F3E08BE00382FB0
:100F80003C080A3C031DD12F3B0BD12FB709B809F0
:100F9000B909BA09B70A0319B80A0319B90A031932
:100FA000BA0A3708F7003808F8003908F9003A0893
:100FB000FA000313003403176208F80161020318F2
:100FC000E42F6108F700F02FF7010830E300E10D8E
:100FD000F70D620877020318F700F80DE30BE72F0F
:100FE000031300348C1EF62F4620F22F8316861230
:100FF00083128612003483168612831286160034FA
:101000000317BC010408BB003C10831B3C14350EC5
:10101000F038B700B707E23EB800323EBA003508F4
:101020000F39B807B807BA07E93EB900B907B907D9
:10103000340E0F39B907BA07B90DBA0DBA09BA0D8E
:1010400034080F39BA07B70D0730B6000A30BA07AF
:10105000B903031C2728B907B803031C2B28B807BA
:10106000B703031C2F28B707B603031C33283630F9
:101070008400831707303B053B1384073A30040292
:1010800003193B170008F700031D4E283B1B4E2891
:101090003B1A6428BB194E2820305128BB153B123F
:1010A0003030F707B5010408B4003510831B351440
:1010B0007708E3008A110313B9248A15031734084B
:1010C0008400831335188317840A3B1F3E280313BB
:1010D0000034780803175F08E1006430E2008A11E9
:1010E0000313DB278A1577080317DF0078083030F1
:1010F000031D8128E01C8C28E0198C28601A203000
:101100008428E01160126014F8077808E3008A115F
:101110000313B9248A1503175F08E1000A30E200BF
:101120008A110313DB278A1577080317DF00780875
:101130003030031DA128E019A928601CA928601AD5
:101140002030F8077808E3008A110313B9248A15C0
:1011500003173030DF075F08E3008A110313B92457
:101160008A1500340317E21BC9280F30F700610EFF
:10117000F7050A3077020318C0283030F707C22875
:101180006208F7077708E3008A110313B9248A1568
:1011900003170F30E1050A3061020318D1283030FF
:1011A000D328E2136208E1076108E3008A11031300
:1011B000B9248A1500340317DF080319E82803133C
:1011C0003C10BC103C11BC113C12BC12BD100317EA
:1011D00003133C13BC133D103D1100341C30831627
:1011E000D0008A1183123E2B8A1564008316141CCA
:1011F000E62C831213088316D000500B5F290830A9
:10120000F80083121F08C73978049F0086148316DC
:1012100086100130031790008A11831203133424BF
:101220008A150F300317B500D030B4008A110313AC
:101230004C248A15861083168610831241080317E2
:10124000C400031340080317C30003133F08031728
:10125000C20003133E080317C100C801C7010330D1
:10126000C600E830C5008A110313E4218A157A0804
:10127000031793007908920078089100770890008E
:101280000313EE01D130ED0005308400031713087D
:10129000B7001208B6001108B5001008B4000330FA
:1012A000B8008A110313C8248A150317B501D13079
:1012B000B4008A11031341258A15E52C83165008C2
:1012C000023C031DC3290830F80083121F08C739E8
:1012D00078049F000615831606110130031790004D
:1012E0008A118312031334248A150F300317B500B3
:1012F000D030B4008A1103134C248A1506118316CA
:101300000611831241080317C40003134008031792
:10131000C30003133F080317C20003133E0803175B
:10132000C100C801C7010330C600E830C5008A11FA
:101330000313E4218A157A080317930079089200B1
:1013400078089100770890000313EE01D130ED008A
:101350000530840003171308B7001208B6001108FF
:10136000B5001008B4000330B8008A110313C82474
:101370008A150317B501D130B4008A110313412532
:101380008A15E52C83165008033C031D272A0830D4
:10139000F80083121F08C73978049F00861583164A
:1013A00086110130031790008A118312031334242D
:1013B0008A150F300317B500D030B4008A1103131B
:1013C0004C248A158611831686118312410803174F
:1013D000C400031340080317C30003133F08031797
:1013E000C20003133E080317C100C801C701033040
:1013F000C600E830C5008A110313E4218A157A0873
:1014000003179300790892007808910077089000FC
:101410000313EE01D130ED000530840003171308EB
:10142000B7001208B6001108B5001008B400033068
:10143000B8008A110313C8248A150317B501D130E7
:10144000B4008A11031341258A15E52C8316500830
:10145000043C031D8B2A0830F80083121F08C7398B
:1014600078049F00061683160612013003179000B9
:101470008A118312031334248A150F300317B50021
:10148000D030B4008A1103134C248A150612831637
:101490000612831241080317C40003134008031700
:1014A000C30003133F080317C20003133E080317CA
:1014B000C100C801C7010330C600E830C5008A1169
:1014C0000313E4218A157A08031793007908920020
:1014D00078089100770890000313EE01D130ED00F9
:1014E0000530840003171308B7001208B60011086E
:1014F000B5001008B4000330B8008A110313C824E3
:101500008A150317B501D130B4008A1103134125A0
:101510008A15E52C83165008323C031DC22A003080
:10152000F80083121F08C73978049F000317B5011C
:101530000C30B4008A1103134C248A15EE01D1300B
:10154000ED000530840041080317B700031340087D
:101550000317B60003133F080317B50003133E0833
:101560000317B4000330B8008A110313C8248A1586
:101570000317B501D130B4008A11031341258A1530
:10158000E52C83165008333C031DFF2A2030F80059
:1015900083121F08C73978049F0010300317B50065
:1015A000B401B700B601C830B8000530B9008A11DF
:1015B00003136C258A15EE01D130ED00053084004F
:1015C00041080317B700031340080317B6000313BD
:1015D0003F080317B50003133E080317B400033098
:1015E000B8008A110313C8248A150317B501D13036
:1015F000B4008A11031341258A15E52C831650087F
:101600003C3C031D522B831203179101DC309000E8
:101610008A11031349268A150317B601DC30B50079
:101620008A1103136D268A157808B0007708AF0079
:10163000EE01D130ED001030840030080317B50002
:1016400003132F080317B400031300200317B50179
:10165000D130B4008A11031341258A158A11B322AF
:101660008A150317B401031330080317B6000313D8
:101670002F080317B5008A110313A2218A15031737
:10168000B4018A1103136F218A157908FA007808CA
:101690002F02031D4F2B7A0830020319502B3C14E4
:1016A000E52C831650083D3C031DA72B831203171E
:1016B0009101DC3090008A11031349268A15031723
:1016C000B601DC30B5008A1103136D268A1578083F
:1016D000B2007708B100EE01D130ED001030840087
:1016E00032080317B500031331080317B4000313BE
:1016F00000200317B501D130B4008A11031341252E
:101700008A158A1128228A1502300317B4000313A0
:1017100032080317B600031331080317B5008A1106
:101720000313A2218A1502300317B4008A11031390
:101730006F218A157908FA0078083102031DA42B5D
:101740007A0832020319A52B3C14E52C83165008A5
:101750003E3C031DF92B831203179101DC309000EE
:101760008A11031349268A150317B601DC30B50028
:101770008A1103136D268A157808B4007708B30020
:10178000EE01D130ED001030840034080317B500AD
:10179000031333080317B400031300200317B50124
:1017A000D130B4008A11031341258A150430031780
:1017B000B400031334080317B600031333080317E8
:1017C000B5008A110313A2218A1504300317B4004F
:1017D0008A1103136F218A157908FA0078083302F9
:1017E000031DF62B7A0834020319F72B3C14E52C61
:1017F00083165008463C031D182C8312861283164C
:1018000086128312EE01D130ED0083165008831248
:101810000317DF001B30E000031369200317B50135
:10182000D130B4008A11031341258A15E52C8316A3
:101830005008473C031D372C8312861683168612E8
:101840008312EE01D130ED00831650088312031786
:10185000DF001B30E000031369200317B501D1300E
:10186000B4008A11031341258A15E52C831650080C
:10187000503C031DC72C00308312BC1801300317E5
:101880009101003003133C1901300030031711049B
:10189000930000300313BC190130F700770CF701F7
:1018A0000318F71777080317130495000030031384
:1018B0003C1A0130F700F70EF70DF70DC030F705B1
:1018C000770803171504970000300313BC1A013082
:1018D000F700F70EF70DE030F70577080317170448
:1018E0009900003003133C1B0130F700F70EF03075
:1018F000F7057708031719049B0000300313BC1B7E
:101900000130F700F70DF70DF70DF830F705770800
:1019100003171B049D00003003133D180130F7002E
:10192000F70DF70DFC30F705770803171D049F002E
:1019300000300313BD180130F7000310F70D7708CE
:1019400003171F04A100003003133D1901300317D2
:1019500021040313B800B901EE01D130ED003908BC
:101960000317E1003730E2000313B22038080317F1
:10197000E1003730E2000313B2200317B501D13084
:10198000B4008A11031341258A15E52C83165008EB
:10199000513C031DE62C013083120317DF000313B3
:1019A000DB20EE01D130ED008316500883120317BF
:1019B000DF001B30E000031369200317B501D130AD
:1019C000B4008A11031341258A1583168312F52862
:1019D0008A150A16E72E8A11F2278A15E90183165D
:1019E0008C16C03083128B048A150A12352D0F30E5
:1019F00083168500C1308600933087008312EF0084
:101A0000051283160512831285128316851283121E
:101A10008610831686108312061183160611831210
:101A200086118316861183120612831606128312FC
:101A3000861283168612831207116F116F088316A0
:101A4000870083128711EF116F08831687008312B6
:101A50008712EF126F0883168700831207136F1324
:101A60006F08831687008312EB2C9412EF126F0815
:101A70008316870083126F166F0883168700831200
:101A8000EF116F0883168700213083129400003015
:101A9000831694001F1383121F179F1783169F1717
:101AA00083121F1483161F149F101F159F150730D4
:101AB000831203178D0083168C130C1483120C08E9
:101AC000993C031D982DB4018A1103136F218A15C7
:101AD0007908B0007808AF0002300317B4008A110B
:101AE00003136F218A157908B2007808B100043019
:101AF0000317B4008A1103136F218A157908B40003
:101B00007808B300053003178D0083168C130C146E
:101B100083120C080313B500063003178D008316DB
:101B20008C130C1483120C080313B700322E031706
:101B3000B401031330080317B60003132F0803176B
:101B4000B5008A110313A2218A1502300317B400CD
:101B5000031332080317B600031331080317B50047
:101B60008A110313A2218A1504300317B40003134A
:101B700034080317B600031333080317B5008A119E
:101B80000313A2218A1505300317B9000313350882
:101B90000317BA008A11031386218A15063003172A
:101BA000B900031337080317BA008A1103138621FB
:101BB0008A150317B4018A1103136F218A15790856
:101BC000FA0078082F02031D232E7A083002031D25
:101BD000232E02300317B4008A1103136F218A15D4
:101BE0007908FA0078083102031D232E7A083202A0
:101BF000031D232E04300317B4008A1103136F2131
:101C00008A157908FA0078083302031D232E7A0812
:101C10003402031D232E053003178D0083168C1309
:101C20000C1483120C0803133502031D232E0630F7
:101C300003178D0083168C130C1483120C080313E6
:101C400037020319252EBC14322E9930B600073006
:101C50000317B900031336080317BA008A110313D8
:101C600086218A15370B442E061583160611083077
:101C7000031790008A118312031334248A15061166
:101C800083160611522E831286148316861008308E
:101C9000031790008A118312031334248A158610C7
:101CA000831686108312BD1E562EBD148A150A1681
:101CB000052D0317B4080319652E0313E90803194A
:101CC000632E0317652E592E03170313E908031D0E
:101CD0006D2E0030F800922F922F35086C02031DF4
:101CE0008E2F831623083F3C031DFA2E2408403C08
:101CF00003187E2E24085A3C0318862E2408603CC4
:101D00000318FA2E24087A3C031CFA2E2508403CBE
:101D100003188E2E25085A3C0318962E2508603C81
:101D20000318FA2E25087A3C031CFA2E8312EE01C2
:101D30007130ED008316230883120317E3008A1124
:101D40000313B9248A158316240883120317E300AA
:101D50008A110313B9248A158316250883120317E1
:101D6000E3008A110313B9248A1583162408463C1C
:101D7000031DBE2E2508433C0319C62E2408663CCD
:101D8000031DF22E2508633C031DF22E26082F3C6E
:101D90000318ED2E2608393C031CED2E8312EE01AC
:101DA000AC30ED008316260883120317E3008A1176
:101DB0000313B9248A150317B601AC30B5008A1194
:101DC00003136D268A157A088316B9007908B800BE
:101DD0007808B7007708B600F22EFF30B900B800D7
:101DE000B700B6008312E901E6160130F800922F21
:101DF0008D2F83162308403C0318022F23085A3CDA
:101E000003180A2F2308603C0318892F23087A3C03
:101E1000031C892F2408403C0318122F24085A3C25
:101E200003181A2F2408603C0318892F24087A3CD1
:101E3000031C892F8312EE017130ED0083162308F5
:101E400083120317E3008A110313B9248A1583163A
:101E5000240883120317E3008A110313B9248A1597
:101E6000831625082F3C03187C2F2508393C031CBA
:101E70007C2F8312EE01AC30ED008316250883120F
:101E80000317E3008A110313B9248A158316260861
:101E900083120317E3008A110313B9248A158316EA
:101EA000270883120317E3008A110313B9248A1544
:101EB0008316280883120317E3008A110313B92439
:101EC0008A158316290883120317E3008A11031366
:101ED000B9248A150317B601AC30B5008A11031373
:101EE0006D268A157A088316B9007908B800780833
:101EF000B7007708B600812FFF30B900B800B700EF
:101F0000B6008312E901E6120130F800922F8D2FFE
:101F100083160030F8008312922F922FE9010030CF
:101F2000F800922F8A150A160C2DBD1BA52F061638
:101F3000831606128312BD1796308316031790007E
:101F40008A118312031334248A1500340317E10124
:101F500061085F0784008313601883170313130855
:101F600093018316141CB22F831213088000003AC9
:101F70000319C92F031761080A3C0318C12F031363
:101F8000C92FE10A6400A630F700F70BC52FA82F70
:101F9000031300346618D12F06128316061283121B
:101FA000BD130034831603174608C8004508CA004D
:101FB0004408C9004708003C0318F32F4A08FA00F8
:101FC0004908840083137A18831748080002031D08
:101FD000EE2F4908F8004A08F900F62FC90A03193C
:101FE000CA0AC703DA2F0030F800F900831203137E
:0A1FF0000034F92F8A150A16EC2EB2
:1020000003173508FA003408840083137A188317FD
:102010000008B8003708FA003608840083137A18DD
:10202000831700083802031971283508FA003408AC
:10203000840083137A1883170008B9003908403CDC
:102040000318262839085A3C03182E283908603C02
:102050000318882839087A3C031C88283708FA00B6
:102060003608840083137A1883170008BA003A08E8
:10207000403C03183F283A085A3C031847283A08BE
:10208000603C031888283A087A3C031C88283508E5
:10209000FA003408840083137A1883170008BB0001
:1020A0003708FA003608840083137A188317203023
:1020B00000073B02031971283708FA00360884002C
:1020C00083137A1883170008BD003508FA00340816
:1020D000840083137A188317203000073D02031D04
:1020E00088283508FA003408840083137A18831787
:1020F0008008031D7E280030F800A1283508FA006A
:102100003408B40A0319B50AB60A0319B70A012834
:102110003508FA0034088400831335188317000843
:10212000B8003708FA00360884008313371883177D
:102130000008380203189F28FF30FA00A028013059
:10214000F80003130034103083160317C800F7019A
:10215000FA01C50CC40C031CB3284608F707031882
:10216000FA0A4708FA07FA0CF70CF90CF80CC80B36
:10217000A928031383128A110A16312B0A12FB278E
:102180000A160317E101E0016108013C031CE8287D
:10219000031DCE286008903C031CE8280313EF17AA
:1021A0006F08831687008312871BDB280317E10162
:1021B000E001E128031364001030F700F70BDE287C
:1021C0000317DF08031D6400E00A0319E10AC428AD
:1021D0000A120313F2270A168A110A16A42C0C1EDF
:1021E000EF2803176708031399008A110A161829A4
:1021F000031765100A120313FB270A160317E201DF
:102200006208043C031C3A29031368130317E30113
:102210005F08630203181E296108FA006008840041
:102220008313611883170008E600E7000313EF2803
:102230000317E00A0319E10AE30A08290313681BDC
:102240002E2964088316031790000A1283120313C1
:1022500034240A16031765143A29031364088316F5
:10226000031790000A128312031334240A1603176B
:10227000E20A00290A120313F2270A160030031794
:1022800065180130F80003138A110A16AD2CBD1F22
:10229000AB2B1308503093008316141C4D29323099
:1022A000031790000A128312031334240A1603172B
:1022B000E001BA30DF000A128A150313A6270A16B6
:1022C0008A11831603179101BA3090001108930008
:1022D000100892001308FA001208840083137A1879
:1022E0008317800803197829920A0319930A6A2927
:1022F00010081202F7001308FA001108031C110F4E
:10230000FA027708F8007A08F9007908910078084D
:1023100090009108031D90291008033C0318A82B76
:102320009101BA30900093019201103094009B010A
:102330009C0130309E0031309F003230A00033309D
:10234000A1003430A2003530A3003630A40037306D
:10235000A5003830A6003930A7006130A8006230EF
:10236000A9006330AA006430AB006530AC00663071
:10237000AD006730AE006830AF006930B0006A3041
:10238000B1006B30B2006C30B3006D30B4006E3011
:10239000B5006F30B6007030B7007130B8007330E0
:1023A000B9007430BA007530BB007630BC007730AD
:1023B000BD007830BE007930BF007A30C000C10166
:1023C00011089600100895001608FA0015088400F8
:1023D00083137A1883170008203C031DF329950AFC
:1023E0000319960AE4291608FA00150884008313D5
:1023F0001618831700082D3C0319092A1608FA003D
:102400001508840083131618831700082B3C031D3E
:10241000152A1608FA001508950A0319960A840069
:1024200083137A1883170008162A2B309D001D0885
:102430002D3C031D2A2A120813040319262A120808
:102440008400831313188317100880000030F800ED
:10245000F9009F2B941B352A140B2F2A352A941B25
:10246000452A1408243C0318452A120813040319AA
:10247000402A120884008313131883171008800061
:102480000030F800F9009F2BDB2A94080319A02ADA
:102490001408103C031D6F2A1608FA001508840062
:1024A00083137A1883170008303C031D6F2A01300C
:1024B000150784008313161883170008783C031946
:1024C0006B2A013015078400831316188317000840
:1024D000583C031D6F2A023095070318960A14080A
:1024E000083C031D822A1608FA001508840083138D
:1024F0007A1883170008303C031D822A01309507A3
:102500000318960A1408023C031D9F2A1608FA00B5
:102510001508840083137A1883170008303C031DC4
:102520009F2A0130150784008313161883170008AB
:10253000623C031D9F2A023095070318960ADB2A86
:102540001608FA001508840083137A188317000808
:10255000303C0319AE2A0A309400DB2A01301507FB
:1025600084008313161883170008783C0319C22AC5
:102570000130150784008313161883170008583C90
:10258000031DC92A10309400023095070318960ADB
:10259000DB2A0130150784008313161883170008FF
:1025A000623C031DD92A0230940095070318960A4D
:1025B000DB2A0830940016089800150897001608C2
:1025C000FA001508840083137A1883170008303C3A
:1025D000031DEE2A950A0319960ADF2A1608FA0047
:1025E000150884008313161883170008C200403CA6
:1025F0000318012B42085A3C031C012B42082038C7
:10260000022B4208C3000130C5009E30C4004208BE
:10261000C6001408C7000A128A1583120313D227B2
:102620000A168A117908831603179A007808990008
:102630009908031D1E2B9A080319792BFA01140817
:10264000F700941BFA03C2007A08C3001C08C500F7
:102650001B08C4004308C7004208C60083120313C6
:10266000A328790883160317C4007808C3009E3096
:102670001902F7001A08FA000130031C0230FA02AE
:1026800077084307F80044080318440FFA0778084E
:102690009B007A089C00950A0319960A1608FA000E
:1026A000150884008313161883170008C200403CE5
:1026B0000318612B42085A3C031C612B4208203846
:1026C000622B4208C3000130C5009E30C40042089E
:1026D000C6001408C7000A128A1583120313D227F2
:1026E0000A168A117908831603179A007808990048
:1026F000182B15081702031D902B16081802031D2E
:10270000902B1208130403198C2B120884008313D6
:1027100013188317100880000030F800F9009F2B71
:102720001208130403199B2B120884008313131837
:102730008317150880001B08F8001C08F9007908A9
:1027400083120313BB007808BA00AB2B8316031760
:10275000831203133D1500303C1801308316031714
:102760009101003083120313BC180130003083162E
:102770000317110493000030831203133C19013036
:1027800000308316031713049500003083120313DF
:10279000BC190130F700770CF7010318F717770819
:1027A00083160317150497000030831203133C1A95
:1027B0000130F700F70EF70DF70DC030F705770879
:1027C0008316031717049900003083120313BC1AF1
:1027D0000130F700F70EF70DE030F70577088316A4
:1027E000031719049B000030831203133C1B0130B4
:1027F000F700F70EF030F7057708831603171B0470
:102800009D00003083120313BC1B0130F700F70D4D
:10281000F70DF70DF830F7057708831603171D0439
:102820009F000030831203133D180130F700F70DAD
:10283000F70DFC30F7057708831603171F04A10076
:10284000003083120313BD180130F7000310F70D99
:102850007708831603172104A300003083120313A3
:102860003D19013083160317230483120313B800A4
:10287000B9013A08B8043B08B9040130EE0037301A
:10288000ED002A300317E3000A120313B9240A16D5
:1028900035080317DF000130E0000A128A15031320
:1028A00069200A168A110317340884008313351827
:1028B0008317003000040319712CE0010408DF00C5
:1028C0006010831B60140008E3000A120313B9248C
:1028D0000A1603175F088400831360188317840A9D
:1028E000592C031339080317E1003730E2000A12AC
:1028F0008A150313B2200A168A1138080317E1005B
:102900003730E2000A128A150313B2200A168A1120
:102910000D300317E3000A120313B9240A160A3014
:102920000317E3000A120313B9240A160317B601AA
:10293000373036078400831780080319A12CB60AA4
:10294000982CDF010313BE2803173608DF0001307F
:10295000E1003730E0000313F828F808031DBA2C13
:102960000A308316031790000A12831203133424CB
:102970000A16A42C0317DF010A128A150313DB20A1
:102980000A168A1100348316B608031D182DB708DD
:10299000031D182DB808031D182DB908031D182D87
:1029A0000A128A15831295270A168A1113084630CF
:1029B00093008316141CDA2C3230031790000A128D
:1029C0008312031334240A160317E001BA30DF0020
:1029D0000A128A150313A6270A168A110317B601CD
:1029E000BA30B5000A1203136D260A167A080317C7
:1029F000B7007908B6007808B5007708B400463CFF
:102A0000031D0B2DB508031D0B2DB608031D0B2D43
:102A1000B70803190F2D03133D15162D03170313C4
:102A200066100A128A15CA270A168A11802D831683
:102A3000360B7E2DB708031D7E2DB808031D7E2D95
:102A4000B908031D7E2D8312061683160612831203
:102A5000BD1702300317B4009630831690000A1297
:102A60008312031334240A160317B40B2C2D0313FB
:102A70001308473093008316141C3C2D3230031783
:102A800090000A128312031334240A160317E0017C
:102A9000BA30DF000A128A150313A6270A168A1114
:102AA0000317B601BA30B5000A1203136D260A16D1
:102AB0007A080317B7007908B6007808B5007708D8
:102AC000B400473C031D6D2DB508031D6D2DB608E0
:102AD000031D6D2DB7080319712D03133D157C2DB2
:102AE00003170313661419308316031790000A1294
:102AF0008312031334240A16802D83168312BC1705
:102B00000317B501B401031347218A150A16212DB5
:102B10008316B608031DA82DB708031DA82DB808F5
:102B2000031DA82DB908031DA82D83128614831632
:102B300086100830031790000A12831203133424FE
:102B40000A168610831686108312B701C92D8316C4
:102B5000360BC72DB708031DC72DB808031DC72D99
:102B6000B908031DC72D83120615831606110830F8
:102B7000031790000A128312031334240A16061155
:102B80008316061101308312B700C92D83168312F4
:102B9000BC1706300317B900031337080317BA0030
:102BA0000A12031386210A16063003178D008316B6
:102BB0008C130C1483120C08031337020319E12D34
:102BC000BC140317B501B401031347218A150A1673
:102BD000332D8316B608031DFA2DB708031DFA2DF1
:102BE000B808031DFA2DB908031DFA2D8312E6104B
:102BF0000B2E8316360B092EB708031D092EB808B5
:102C0000031D092EB908031D092E8312E6140B2E8D
:102C100083168312BC170317B501B40103134721B0
:102C20008A150A16452D0A128A1595270A168A1141
:102C30001308513093008316141C1C2E32300317D6
:102C400090000A128312031334240A160317E001BA
:102C5000BA30DF000A128A150313A6270A168A1152
:102C60000317B601BA30B5000A1203136D260A160F
:102C70007A080317B7007908B6007808B500770816
:102C8000B400513C031D4D2EB508031D4D2EB60852
:102C9000031D4D2EB7080319512E03133D15592E50
:102CA00003170130DF000A128A150313DB200A160E
:102CB0008A110317B501B401031347210A128A15BB
:102CC000CA270A168A118A150A16572D07156F1179
:102CD0006F08831687000030F80083121F08C73979
:102CE00078049F0009308316031790000A1283129C
:102CF000031334240A160317B5011930B4000A125D
:102D000003134C240A1607116F116F0883168700EE
:102D10008312EE014630ED000530840041080317B0
:102D2000B700031340080317B60003133F08031747
:102D3000B50003133E080317B4000330B8000A12AD
:102D40000313C8240A160317B5014630B400031351
:102D500047218A150A16692D0A128A1595270A161F
:102D60008A111308323093008316141CB52E3230AA
:102D7000031790000A128312031334240A16031750
:102D8000E001BA30DF000A128A150313A6270A16DB
:102D90008A110A128A15CA270A168A11EE014630CC
:102DA000ED00BA3084008313003000040319EE2EC6
:102DB0000317B5010408B4003510831B351400084F
:102DC000E3000A120313B9240A1603173408840017
:102DD000831335188317840A0313D42E0317B50100
:102DE0004630B400031347218A150A167B2D0715B8
:102DF0006F116F08831687000830F80083121F08D0
:102E0000C73978049F0009308316031790000A120F
:102E10008312031334240A1610300317B500B401CB
:102E2000B700B601C830B8000530B9000A12031364
:102E30006C250A1607116F116F088316870083121D
:102E4000EE014630ED000530840041080317B7005D
:102E5000031340080317B60003133F080317B50018
:102E600003133E080317B4000330B8000A1203131B
:102E7000C8240A160317B5014630B40003134721CE
:102E80008A150A168D2D0A128A1595270A168A1197
:102E90001308333093008316141C4C2F3230031761
:102EA00090000A128312031334240A160317E00158
:102EB000BA30DF000A128A150313A6270A168A11F0
:102EC000EE014630ED00BA30840083130030000478
:102ED0000319802F0317B5010408B4003510831BB4
:102EE00035140008E3000A120313B9240A16031765
:102EF00034088400831335188317840A0313662F5C
:102F00000317B5014630B400031347210A128A158E
:102F1000CA270A168A118A150A169F2DEE01463015
:102F2000ED001030840030080317B50003132F089C
:102F30000317B4000A128A15031300200A168A1117
:102F40000317B5014630B400031347218A150A164A
:102F5000C22DEE014630ED00103084003208031718
:102F6000B500031331080317B4000A128A150313BE
:102F700000200A168A110317B5014630B400031366
:102F800047218A150A16D52DEE014630ED00103086
:102F9000840034080317B500031333080317B40083
:102FA0000A128A15031300200A168A110317B501A5
:102FB0004630B400031347218A150A16E82DEE01A6
:102FC0004630ED0037080317DF001B30E0000A121F
:102FD0008A15031369200A168A110317B5014630B2
:102FE000B400031347218A150A16FB2D0317B501F8
:0C2FF000B401031347218A150A160E2EA7
:103000008316B908031D8028B808031D8028B70857
:10301000031D80283608033C031C80280A128312F3
:1030200095270A1601308316360783120317B4005A
:1030300083160313370883120317B50000300318F3
:103040000130B50783160313380883120317B6003F
:10305000003003180130B6078316031339088312B2
:103060000317B700003003180130B7070313130824
:1030700003173408031393008316141C3D283230C1
:10308000031790000A128A118312031334240A16BC
:103090008A150317E001BA30DF000A120313A627CE
:1030A0000A16EE014630ED00BA308400831300307A
:1030B0000004031973280317B5010408B400351080
:1030C000831B35140008E3000A128A110313B92484
:1030D0000A168A15031734088400831335188317DA
:1030E000840A031357280317B5014630B4008A1128
:1030F000031347218A150A12CA270A16892883163C
:103100008312BC170317B501B4018A1103134721B9
:103110008A158A150A16B02DEE014630ED00031708
:10312000B40134080A128A1103133E200A168A15C4
:1031300000380319A7280317B40AE3000A128A11FA
:103140000313B9240A168A150317912803130317CA
:10315000B5014630B4008A11031347218A158A1538
:103160000A16202E04080317B8003B30BF009A301F
:10317000BE00CA30BD00BC010A30BA003708C40026
:103180003608C3003508C2003408C1003F08C80033
:103190003E08C7003D08C6003C08C5000A128A1157
:1031A0000313E4210A168A1500080317B400840AE1
:1031B0000008B500840A0008B600840A0008B700B9
:1031C000F708031DF6283A08013A0319F6283808CB
:1031D0000319F7280F393A020319F02803180229B6
:1031E000B81B0229381BF7282030F828B8013030E6
:1031F000F7077708E3000A128A110313B9240A16A5
:103200008A1503173F08C4003E08C3003D08C200EA
:103210003C08C100C801C701C6010A30C5000A1236
:103220008A110313E4210A168A157A080317BF00CE
:103230007908BE007808BD007708BC00BA0BBE282C
:10324000031300348316B908031D332AB808031D7D
:10325000332A3708273C031C332A031D3329360839
:10326000103C031C332A0A12831295270A161308EE
:103270003C3093008316141C3B298312EE01C530A9
:10328000ED00413084008316390883120317B7001C
:1032900083160313380883120317B600831603132B
:1032A000370883120317B5008316031336088312F9
:1032B0000317B4000313B22020300317E3000A12EF
:1032C0008A110313B9240A168A150317B501C530EC
:1032D000B4000A128A11031341250A168A153230E6
:1032E0008316031790000A128A11831203133424E1
:1032F0000A168A150317E001BA30DF000A12031319
:10330000A6270A1603308316031790000A128A11A3
:103310008312031334240A168A150317B601BA3030
:10332000B5000A128A1103136D260A168A157A0847
:103330000317B7007908B6007808B5007708B4001D
:10334000831603133608831203173402031D062A5B
:10335000831603133708831203173502031D062A49
:10336000831603133808831203173602031D062A37
:10337000831603133908831203173702031D062A25
:103380008316031337088312B0008316360883129E
:10339000AF000317B401031330080317B60003137B
:1033A0002F080317B5000A128A110313A2210A1667
:1033B0008A150317B4010A128A1103136F210A1622
:1033C0008A157908FA0078082F02031DEB297A087C
:1033D00030020319EC29BC14EE014630ED00103028
:1033E000840030080317B50003132F080317B40037
:1033F0000A12031300200A160317B5014630B40061
:103400008A11031347218A152E2A031703133D152A
:10341000EE014630ED0041308400831639088312F6
:103420000317B70083160313380883120317B60077
:1034300083160313370883120317B500831603138B
:10344000360883120317B4000313B2200317B50123
:103450004630B4008A11031347218A150A12CA277D
:103460000A163C2A83168312BC170317B501B40150
:103470008A11031347218A158A150A16312E8316DD
:10348000B908031D332BB808031D332B3708273C1D
:10349000031C332B031D502A3608103C031C332B0E
:1034A0000A12831295270A1613083D3093008316DB
:1034B000141C582A8312EE01C530ED0041308400FF
:1034C0008316390883120317B700831603133808CD
:1034D00083120317B60083160313370883120317EA
:1034E000B50083160313360883120317B4000313C1
:1034F000B22020300317E3000A128A110313B92403
:103500000A168A150317B501C530B4000A128A11CC
:10351000031341250A168A153230831603179000CB
:103520000A128A118312031334240A168A15031708
:10353000E001BA30DF000A120313A6270A1603308F
:103540008316031790000A128A118312031334247E
:103550000A168A150317B601BA30B5000A128A1185
:1035600003136D260A168A157A080317B70079081F
:10357000B6007808B5007708B40083160313360840
:10358000831203173402031D252B831603133708F8
:10359000831203173502031D252B831603133808E6
:1035A000831203173602031D252B831603133908D4
:1035B000831203173702031D252B831603133708C5
:1035C0008312B200831636088312B100023003174B
:1035D000B400031332080317B600031331080317AE
:1035E000B5000A128A110313A2210A168A150230A5
:1035F0000317B4000A128A1103136F210A168A15E1
:103600007908FA0078083102031D0A2B7A08320281
:1036100003190B2BBC14EE014630ED001030840072
:1036200032080317B500031331080317B4000A1258
:10363000031300200A160317B5014630B4008A119F
:10364000031347218A152E2B031703133D15031768
:10365000B501B4018A11031347218A150A12CA273A
:103660000A163C2B83168312BC170317B501B4014D
:103670008A11031347218A158A150A16422E8316CA
:10368000B908031D282CB808031D282C3708273C2F
:10369000031C282C031D502B3608103C031C282C1F
:1036A0000A12831295270A1613083E3093008316D8
:1036B000141C582B8312EE01C530ED0041308400FC
:1036C0008316390883120317B700831603133808CB
:1036D00083120317B60083160313370883120317E8
:1036E000B50083160313360883120317B4000313BF
:1036F000B22020300317E3000A128A110313B92401
:103700000A168A150317B501C530B4000A128A11CA
:10371000031341250A168A153230831603179000C9
:103720000A128A118312031334240A168A15031706
:10373000E001BA30DF000A120313A6270A160317A6
:10374000B601BA30B5000A128A1103136D260A16A3
:103750008A157A080317B7007908B6007808B5000B
:103760007708B40083160313360883120317340254
:10377000031D1A2C8316031337088312031735020F
:10378000031D1A2C831603133808831203173602FD
:10379000031D1A2C831603133908831203173702EB
:1037A000031D1A2C8316031337088312B4008316E3
:1037B00036088312B30004300317B400031334082F
:1037C0000317B600031333080317B5000A128A1152
:1037D0000313A2210A168A1504300317B4000A1233
:1037E0008A1103136F210A168A157908FA007808DE
:1037F0003302031DFF2B7A0834020319002CBC147A
:10380000EE014630ED001030840034080317B50097
:10381000031333080317B4000A12031300200A1617
:103820000317B5014630B4008A11031347218A15E6
:10383000232C031703133D150317B501B4018A1197
:10384000031347218A150A12CA270A16312C831638
:103850008312BC170317B501B4018A110313472162
:103860008A158A150A16532E8316B908031D612C72
:10387000B808031D612CB708031D612C3608633C92
:10388000031C612C36088312B50005300317B900FC
:10389000031335080317BA000A128A11031386218D
:1038A0000A168A15053003178D0083168C130C1425
:1038B00083120C080313350203195F2CBC14632C0C
:1038C00083168312BC17EE014630ED0041308400B0
:1038D0008316390883120317B700831603133808B9
:1038E00083120317B60083160313370883120317D6
:1038F000B50083160313360883120317B4000313AD
:10390000B2200317B5014630B4008A1103134721D2
:103910008A158A150A16642E4C308316D00044305E
:10392000D100D2014330D3005230D400D5015330FE
:10393000D6004530D700D8014330D9004530DA00F1
:10394000DB013F30DC004230DD005630DE00DF01BD
:103950003F30E0004C30E1005630E200E3013F3000
:10396000E4004230E5004330E600E7013F30E80084
:103970004C30E9004330EA00EB013F30EC004630C8
:10398000ED004330EE00EF013F308312031790004B
:10399000533091004F30920093013F3094005330E8
:1039A0009500960097013F309800543099005030B0
:1039B0009A009B013F309C0043309D0052309E0096
:1039C0009F013F30A0005330A1004E30A200A30160
:1039D0003F30A4005630A5005230A600A701533056
:1039E000A8004F30A900AA015330AB00AC00AD01D4
:1039F0005430AE005030AF00B0015330B1004E3003
:103A0000B200B3010A120313F72C0A16640003175D
:103A1000B4010A120313592E0A16F80803196E2E60
:103A20003D160317B5017130B400B701D030B600B0
:103A30008A11031300208A15F808031D232D8A110B
:103A4000C32C8A156E2E0317B5017130B400B7016F
:103A5000D330B6008A11031300208A15F808031D1D
:103A6000352D8A11882D8A156E2E0317B5017130F8
:103A7000B400B701D630B6008A11031300208A15AE
:103A8000F808031D472D8A11E92D8A156E2E03179C
:103A9000B5017130B400B701D930B6008A110313F3
:103AA00000208A15F808031D592D8A11132E8A1536
:103AB0006E2E0317B5017130B400B701DC30B600CB
:103AC0008A11031300208A15F808031D6B2D8A1133
:103AD000662E8A156E2E0317B5017130B400B7013A
:103AE000E030B6008A11031300208A15F808031D80
:103AF0007D2D8A11AC2E8A156E2E0317B5017130FB
:103B0000B400B701E430B6008A11031300208A150F
:103B1000F808031D8F2D8A11F72E8A156E2E0317B4
:103B2000B5017130B400B701E830B6008A11031353
:103B300000208A15F808031DA12D8A11432F8A152C
:103B40006E2E0317B5017130B400B701EC30B6002A
:103B50008A11031300208A15F808031DB12D0028CF
:103B60006E2E0317B5017130B4000130B70010306C
:103B7000B6008A11031300208A15F808031DC42D0E
:103B80008A118E2F8A156E2E0317B5017130B4007D
:103B90000130B7001430B6008A11031300208A15D3
:103BA000F808031DD72D8A11A92F8A156E2E031729
:103BB000B5017130B4000130B7001830B6008A1179
:103BC000031300208A15F808031DEA2D8A11C42F5B
:103BD0008A156E2E0317B5017130B4000130B7009D
:103BE0001C30B6008A11031300208A15F808031D43
:103BF000FD2D8A11DF2F8A156E2E0317B501713046
:103C0000B4000130B7002030B6008A110313002041
:103C10008A15F808031D102E8A11F62F8A156E2EAC
:103C20000317B5017130B4000130B7002430B6007D
:103C30008A11031300208A15F808031D212E8C28F1
:103C40006E2E0317B5017130B4000130B700283073
:103C5000B6008A11031300208A15F808031D322EBE
:103C600022296E2E0317B5017130B4000130B70060
:103C70002B30B6008A11031300208A15F808031DA3
:103C8000432E3F2A6E2E0317B5017130B400013068
:103C9000B7002E30B6008A11031300208A15F808E9
:103CA000031D542E3F2B6E2E0317B5017130B40047
:103CB0000130B7003130B6008A11031300208A1595
:103CC000F808031D652E342C6E2E3C170317B50122
:103CD000B4018A11031347218A153D12062D8A1556
:103CE0000A16EA2E840183131F30830519308316C8
:103CF0009900A630980090308312980083161F1404
:103D00009F141F159F1107309C008312A901AA015F
:103D1000AF01B001B101B201B301B401B501B60107
:103D2000B701B801B901BA01BB013C10BC103C118C
:103D3000BC113C12BC123C13BC133D10BD103D1114
:103D4000BE01BF01C001C101C201C301C401C5015F
:103D50000330E400E501BD153D12BD123D13BD1356
:103D60006610E610E701E801EB01EC016611E611CF
:103D70006612E612ED01EE01FF30EF00030818397C
:103D8000F70083160E08033977040E148E1483157A
:103D90000316033A83120319D42E083A0319D42EBA
:103DA000133A0319D62ED82EBD16D82EBD12D82EF2
:103DB0000A128A114D290A168A156F146F08831684
:103DC00087008312071CE92EBD110A12EE280A167D
:0C3DD000EA2E8C2C0A12F92F0A16ED2E98
:02400E00313748
:00000001FF
